:100000000C94E7020C943A030C943A030C943A03D0
:100010000C943A030C943A030C943A030C943A036C
:100020000C943A030C943A030C9494230C943A03E2
:100030000C946B230C943A030C943A030C943A03FB
:100040000C943A030C943A030C943A030C943A033C
:100050000C943A030C9467260C943A030C943A03DC
:100060000C943A030C943A030C943A030C943A031C
:100070000C943A030C943A030C943A030C943A030C
:100080000C943A030C943A030C943A030C943A03FC
:100090000C943A030C943A030C943A030C943A03EC
:1000A0000C943A030C943A030C943A03737065650C
:1000B000643A2025730A007573625F737461746516
:1000C0003A20253032580A00686F73742E546173D9
:1000D0006B3A2025640A000D0A676574446576440E
:1000E0006573637220000D0A736574436F6E66203A
:1000F000000D0A00424D20636F6E66696775726578
:10010000640D0A000D0A0052504950453A20000D76
:100110000A005345545F49444C453A20000D0A00FB
:100120005345545F50524F544F434F4C3A20000DAB
:100130000A000D0A496E746572666163653A000DC6
:100140000A00624E756D49666163653A000D0A00EA
:100150006249666163654E756D3A000D0A00436E33
:10016000663A000D0A00624E756D45503A004849E6
:10017000445F50524F544F434F4C5F4B4559424F91
:100180004152440D0A000D0A004E433A000D0A0088
:10019000416464723A000D0A0073657441646472CC
:1001A0003A006570696E666F0D0A00424D20496E17
:1001B00069740D0A000D0A0020000D0A0028686904
:1001C00064626F6F742E682920496E74657266616F
:1001D00063653A000D0A0028686964626F6F742EC7
:1001E000682920537472616E6765207265616420AE
:1001F000636F756E743A20000D0A002868696462A6
:100200006F6F742E682920506F6C6C3A000D0A00D5
:1002100028686964626F6F742E6829206570496E62
:10022000666F5B6570496E74657272757074496E45
:10023000496E646578202B20695D2E6D6178506B66
:100240007453697A653D000D0A0028686964626F1D
:100250006F742E6829206570496E666F5B65704902
:100260006E74657272757074496E496E646578203B
:100270002B20695D2E6570416464723D000D0A009B
:1002800028686964626F6F742E682920693D005286
:100290006F6C6C6F766572206572726F723A20694E
:1002A000676E6F7265640D0A000D0A0020253032FA
:1002B0005800696E7075742025643A002E2E2E4603
:1002C00041494C0D0A0042756666657220706F697F
:1002D0006E746572206973204E554C4C210D0A00D6
:1002E0004C45443A20253032580A000A4C6F6F7052
:1002F0002073746172742E0A000A55534220636F92
:100300006E666967757265642E0A000A544D4B3A31
:100310006433666461632F4C5546413A64366137F5
:1003200064662F554853323A3335363036620A0008
:100330000631FF0974A1010975150026FF009520FB
:10034000750881020976150026FF00952075089131
:1003500002C005010906A101050719E029E71500FA
:10036000250195087501810295017508810105082F
:1003700019012905950575019102950175039101F2
:100380000507190029FF150026FF0095067508814D
:1003900000C009023B00020100A032090400000174
:1003A000030101000921110100012240000705811C
:1003B0000308000A090401000103000000092111DB
:1003C0000100012222000705830320000112011011
:1003D0000100000008EDFE5B001508010200013C71
:1003E00003550053004200200074006F00200055A8
:1003F000005300420020006B006500790062006F2E
:1004000000610072006400200063006F006E0076DF
:10041000006500720074006500720000000803545B
:10042000004D004B000000040309047379737465E8
:100430006D3A20253034580A00636F6E73756D6510
:10044000723A20253034580A0000000000040506E6
:100450000708090A0B0C0D0E0F10111213141516B4
:100460001718191A1B1C1D1E1F20212223242526A4
:100470002728292A2B2C2D2E2F3031323334353694
:100480003738393A3B3C3D3E3F4041424344454684
:100490004748494A4B4C4D4E4F5051525354555674
:1004A0005758595A5B5C5D5E5F606162636465A525
:1004B0006768696A6B6C6D6E6F7071727374757654
:1004C0007778797A7B7C7D7EA8A9AA0000008500D8
:1004D0008788898A8B00000000909100000000004E
:1004E000000000000000000000000000000000000C
:1004F00000000000000000000000000000000000FC
:1005000000000000000000000000000000000000EB
:1005100000000000000000000000000000000000DB
:10052000000000000000000000E0E1E2E3E4E5E696
:10053000E7000000000000000000000000000000D4
:100540000000000000000000000A002530325820A2
:10055000006B6579626F6172643A20000D0A0028B1
:100560005553423A3A496E5472616E736665722908
:100570002065702072657175657374656420000D67
:100580000A00285553423A3A496E5472616E7366B6
:100590006572292061646472207265717565737477
:1005A000656420000D0A00285553423A3A496E54BA
:1005B00072616E736665722920536574416464725A
:1005C000657373204661696C65642000792211248B
:1005D0001FBECFEFDAE0DEBFCDBF04B603FE28C0FA
:1005E0008091720590917305A0917405B091750585
:1005F0008730904BA740B04BD9F4109272051092FF
:100600007305109274051092750514BE0FB6F89418
:10061000A8958091600088618093600010926000CE
:100620000FBE1092010810920008E0E0F8E309956F
:1006300011E0A0E0B1E0EAEDFFE402C005900D9208
:10064000A438B107D9F725E0A4E8B1E001C01D92B4
:10065000A237B207E1F712E0C7EED2E004C021975B
:10066000FE010E94E527C63ED107C9F70E94722409
:100670000C94EB270C940000FF93EF93E09184011E
:10068000F0918501309709F00995EF91FF91089558
:10069000FC018591803011F0EFDFFBCF0895FF273B
:1006A000E0E230E247FF0CC0419597FF09C0EDE260
:1006B0006095709580959095611D711D811D911DAE
:1006C00027FF02C0219530E350E2AA27660F771F6B
:1006D000881F991FAA1FA41710F0A41B63955A9591
:1006E000A9F7AA3008F0A95FA05DAF93F395611553
:1006F00071058105910541F7ED3211F4EF93F39502
:10070000F21718F43F93F395FBCF8F91B5DFFA956D
:10071000E1F70895E991F9918591803021F08532D2
:1007200019F0AADFF9CF089520E0E89455915532E9
:10073000C1F3503311F4689455915A3348F450532F
:1007400090F3220F022E220F220F200D250FF4CF3F
:100750000EF4219589919991533619F3533729F164
:10076000533559F1BC0188279927E8945C3621F468
:100770008991999168945591543639F446EF7EF0F9
:1007800077FF0DC08FEF9FEF0AC055374AE039F071
:10079000583540E121F0523642E009F00895FF93C8
:1007A000EF937DDFEF91FF91B7CFFF93EF93FC01C4
:1007B00081918030B9F360DFFBCFFF93EF9368DF67
:1007C000F1CFDF93CF93CDB7DEB72596A3DFCF91DF
:1007D000DF910895FC018BEF94E0958384838BE295
:1007E00091E09183808389E491E093838283138AEB
:1007F000148A158A168A178A118E81E0828B118AD3
:10080000178288E080878CE381871286138684E0D4
:100810008487158616861786A1E5B5E090E080E00E
:100820002D913D91232B41F4880F991FDC01AF5A84
:10083000BA4FED93FC93089501968031910581F7AD
:100840000895E6E8F2E09281891301C012823196A0
:1008500092E0EC38F907B9F70895A8E8B2E0EFEFB5
:1008600090E02D91821751F0EF3F19F4211101C052
:10087000E92F9F5F9630A9F7EF3F09F408950E2EF8
:10088000000CFF0BEA57FD4F82830895E091E503CA
:10089000F091E603309721F00190F081E02D09946A
:1008A00080E00895E8EDF0E080818E7F80831092F3
:1008B000E2001092DA001092E100A0EEB0E08C911C
:1008C00081608C9380818F77808319BCA7EDB0E025
:1008D0008C918E7F8C9380818F7E80831092C80252
:1008E0000895FC018091DD029091DE028617970742
:1008F000A0F06115710529F49091E8009E7790931E
:10090000E80090E06115710551F4911108C08091E3
:10091000E80082FF35C080E00895BC01F2CF8091ED
:10092000DF028823C9F18530C9F18091E80083FD99
:1009300031C08091E80082FDEACF8091E80080FF1D
:10094000E1CF2091F3008091F200322F282F611522
:10095000710519F02830310558F091E02830310543
:1009600009F090E02091E8002E772093E800CACFAC
:1009700081918093F100615071092F5F3F4FE7CF64
:100980008091DF02882341F0853041F08091E800BA
:1009900083FFBDCF81E0089582E0089583E008954C
:1009A0002091E4003091E50085E69091EC0090FF05
:1009B00006C09091E80090FF06C080E008959091F5
:1009C000E80092FDFACF9091DF02992391F09530E3
:1009D00091F09091EB0095FD10C04091E400509192
:1009E000E5002417350709F381509A01F1F684E0F8
:1009F000089582E0089583E0089581E0089580914C
:100A0000D70287FF13C08091E80082FF06C0809163
:100A1000E8008B778093E80004C08091DF028111A9
:100A2000F2CF08958091DF028823D9F38091E80006
:100A300080FFF8CF8091E8008E77ECCF982F9093CD
:100A4000E900242F762F50E0891731F07091EC00E7
:100A50002091ED005091F00021FD07C09F5F97307D
:100A600071F78093E90081E008953091EB003E7FBB
:100A70003093EB003091ED003D7F3093ED003091ED
:100A8000EB0031603093EB007093EC002093ED00AD
:100A90005093F0002091EE0027FDE0CF80E0089514
:100AA000CF92DF92EF92FF920F931F93CF93DF933A
:100AB000C8EDD0E088818F7E8883E7EDF0E080810B
:100AC0008160808384E082BF81E08093C802888156
:100AD0008E7F888302EE10E0F80110821092DA0017
:100AE00081EEC82ED12CF601108288818F77888301
:100AF00088818068888388818F7D888319BC109263
:100B0000DF021092D6021092D5021092D40290EE1B
:100B1000E92EF12CF70180818B7F808388818160B1
:100B2000888342E060E080E00E941E05F60180813B
:100B30008E7F8083F80180818160808380818860DE
:100B40008083F70180818E7F8083888180618883A4
:100B5000DF91CF911F910F91FF90EF90DF90CF9099
:100B600008950895089508958091CB020895CF9334
:100B7000DF93EC018A819B81DC01ED91FC91048083
:100B8000F581E02D6A8509958A85813439F4EA81F9
:100B9000FB81EA58FF4F80818B7F80831A861B86FA
:100BA0001C861D861E861F86188A80E0DF91CF91E5
:100BB000089581E0693009F080E00895FC018285A4
:100BC0000895DF92EF92FF920F931F93CF93DF93DD
:100BD000EC0185E0E62EF12CFE01869FE00DF11D73
:100BE0001124908596FF24C0192F177001E085E02D
:100BF000D82E8FEF800F8F3008F001E0602F70E06B
:100C0000062FD69EF001D79EF00D1124EC0FFD1F8C
:100C100080858695869586958770181701F16F5F98
:100C20007F4F603168F38D81811302C011501D83A5
:100C300085E08E9DF0018F9DF00D1124EC0FFD1FBE
:100C4000108681E0818712862296D783C683DF9142
:100C5000CF911F910F91FF90EF90DF900895CE01FB
:100C60000E94E105C6CFFC0121E0613499F49C01AA
:100C7000255B3F4F61E0AC014E5F5F4F1586668795
:100C800017865487438735962E173F07B9F7FC011F
:100C9000158208953585631729F02F5F3596203129
:100CA000C9F70895622F0C94E105CF93DF93FC01FF
:100CB00067FD12C0283080F4442319F08581873005
:100CC00059F0EF01A1E0B0E08D85882349F111963C
:100CD0002596A031B105C1F780E018C085E08A9F54
:100CE000E0018B9FD00D1124CE0FDF1F442389F02C
:100CF00081E4888785818F5F858325E02A9FC001F5
:100D00002B9F900D1124E80FF91F8085DF91CF9163
:100D1000089581E08887F1CF2770687B622B0FC030
:100D20006623E1F26770660F660F660F4423A1F336
:100D3000606485818F5F85838770687F682B25E07D
:100D40002A9FC0012B9F900D1124E80FF91F608787
:100D5000862FDCCFFC0121E0611102C006960895C8
:100D60003585631739F02F5F35962031C9F790E04C
:100D700080E00895069635E0239F800D911D112493
:100D800008950F931F93CF93DF932115310599F0A9
:100D9000E901042F162F0E94AA06FC0186ED309768
:100DA00029F01283D183C083038380E0DF91CF9148
:100DB0001F910F91089588EDF9CF81E008952FB725
:100DC000F8946091EA037091EB038091EC039091A9
:100DD000ED032FBF0895CF93C091A402C1110BC0A2
:100DE0000E94DF06643C79408105910520F081E096
:100DF0008093A402C1E08C2FCF9108952FB7F8946F
:100E00008091EA039091EB03A091EC03B091ED0384
:100E10002FBF0895EF92FF920F931F93CF93DF930D
:100E2000D82F0FB607FE46C08091DF02843079F0DC
:100E30008091030190E001962091050130E082232A
:100E40009323209104012817190609F0D0C00E94AD
:100E5000EB0681110FC08091030190E00196209173
:100E6000050130E0822393232091040128171906FD
:100E700009F0BDC00E94FE068C01C091E900CF7050
:100E80008091EC0080FD38C080E0C82B83E0809327
:100E9000E90085E0E82E8091EB0085FD08C0809197
:100EA000EB0080FF04C08091EE0087FD45C0CF704D
:100EB000C093E900E09103018E2F90E0019620910C
:100EC000050130E08223932320910401281719069D
:100ED00009F460C08091010190910201E80FF92F9F
:100EE000F11DD083809103018F5F909105018923CB
:100EF0008093030181E074C080E8C7CFE0910101D5
:100F0000F0910201E80FF11D90818F5F20910501A2
:100F10008223809304019093F1008091E80085FD85
:100F20000BC08091E80080FF07C08091E8008E77B9
:100F30008093E800E0920001809104019091030108
:100F4000981751F19091E80095FDD8CF80E02BC023
:100F50001092F10034C08091030190E0019620913D
:100F6000050130E0822393232091040128171906FC
:100F700009F09DCFF0900001FF2009F498CF0E9466
:100F8000FE068017910709F486CFFA94F0920001CB
:100F90008C0181CF80E024C08091E80085FFD6CF0E
:100FA000D093F10081E02091F3009091F200322F74
:100FB000292F232B79F09091E80090FF0BC090919E
:100FC000E80095FDC5CF9091E8009E779093E800EA
:100FD000E0920001882309F4BECFCF70C093E900EE
:100FE000DF91CF911F910F91FF90EF900895E091C5
:100FF000030170CF0E940A0780E0089561387105EF
:1010000011F00C940A0708950F931F93CF93DF9369
:101010008C01C4E0D0E0B80180E30E94FE07219774
:10102000D1F7DF91CF911F910F910895CF93DF9367
:101030006138710569F0009759F0EC01FE01849167
:101040002196882329F060E870E00E94FE07F6CF21
:10105000DF91CF9108950F931F93CF93DF93FC01FE
:101060008B01EA0180819181892B61F460E870E055
:1010700086EC92E00E94160880E0DF91CF911F91EC
:101080000F9108959281992319F128813981232B99
:1010900099F3D8012D913C91D9014C918381682F0E
:1010A000691B770B80819181860F971FDC014C9320
:1010B0008281815082838881998101979983888375
:1010C000D8018D919C91119701968D939C93DACFC5
:1010D0008381828381E0D1CF8F929F92AF92BF9222
:1010E000CF92DF92EF92FF920E94C1264B015C01EA
:1010F00020E030E04AE755E40E9450276B017C0174
:1011000020E030E040E85FE30E948D2687FD30C09C
:1011100020E03FEF4FE757E4C701B6010E944B279D
:101120001816F4F420E030E040E251E4C501B401C7
:101130000E9450270E94922620E931E06115710536
:1011400049F4FF90EF90DF90CF90BF90AF909F90C9
:101150008F900895C9010197F1F761507109EECFA1
:10116000C701B6010E949226CB010197F1F7E9CFA2
:1011700061E070E0F9CFEF92FF920F931F93CF934E
:10118000DF938A01EB017B01E40EF51ECE15DF052E
:1011900021F089910E940A07F9CFC801DF91CF9110
:1011A0001F910F91FF90EF900895862F0E940A07DC
:1011B00081E090E00895089581E090E008958FEF38
:1011C0009FEF089590E080E008953F924F925F92E4
:1011D0006F927F928F929F92AF92BF92CF92DF9247
:1011E000EF92FF920F931F93CF93DF9300D000D025
:1011F000CDB7DEB76C017A8369835C834B8384E06F
:10120000482E360182E1680E711C93E0392E56019A
:10121000A7E0AA0EB11C12E0552453944601B0E198
:101220008B0E911C29813A812115310509F4CDC01D
:10123000F60180A18230F1F0A8F5882309F457C0A7
:10124000813091F7AE014F5F5F4FBE016D5F7F4F01
:10125000C5010E942B08882309F4B7C0D601159652
:10126000ED91FC911697808191968C939197818155
:1012700092968C93F6017682658230A2D601929680
:101280008C919297843011F493961C92F60181A16F
:1012900082508483258136813087278382878187A6
:1012A00040A205C0833051F3843009F0BDCFD60190
:1012B00092968C919297843019F1853009F44BC045
:1012C000823009F075C0AE014F5F5F4FBE016D5FA8
:1012D0007F4FC5010E942B08882309F476C0F601D0
:1012E000858984A3F6019682858210A29BCF148300
:1012F00085819681908787831287118750A2A2CF1C
:10130000AE014F5F5F4FBE016D5F7F4FC5010E9411
:101310002B08882309F459C0D60155968C9155970E
:10132000833001F756968C9156978130D9F698966E
:101330009C91989757968C91992351F0882391F21C
:10134000F60153A2928996A3938997A385A3CACF46
:10135000813041F6F5CFAE014F5F5F4FBE016D5F4B
:101360007F4FC5010E942B08882379F1D6019396FF
:101370008C919397882309F4B5CF12968D919C9107
:10138000009709F4AFCFDC01ED91FC910190F08161
:10139000E02D7401D60195960C91959797962C9116
:1013A000979796964C91969794966C9109959ACFAB
:1013B000F60185858823F9F0813041F1D6011E962A
:1013C0008D919C91892B09F48DCF0F900F900F90E8
:1013D0000F90DF91CF911F910F91FF90EF90DF90D1
:1013E000CF90BF90AF909F908F907F906F905F90C5
:1013F0004F903F90089591968C9191978250990BC0
:101400001F969C938E931E971D965C9229813A811C
:101410008B819C81782F692FF60146855785411570
:10142000510581F001962115310539F041505109DE
:101430005787468721503109EDCF1A8219827B8365
:101440006C83BCCF3A8329839C838B831586B6CF6C
:1014500008950F931F93CF93C82F8B01282F30E04F
:1014600084E0359527958A95E1F780E3820F8A33EA
:1014700010F087E3820FB8010E94FE07CF7080E36F
:101480008C0F8A3310F087E38C0FB801CF911F9136
:101490000F910C94FE07EF92FF92CF93DF93FC0124
:1014A000E7018289823021F16787408B9B819370AD
:1014B0009330F1F49A8197FF1BC02E81308D321743
:1014C00008F4208F282F30E0D901AA0FBB1FA20FEC
:1014D000B31FAE0FBF1F9F7017969C9317979C81E9
:1014E00018969C93189794E019969C938F5F828B23
:1014F000DF91CF91FF90EF900895EF92FF920F93BD
:1015000002970E944B0A0F91FF90EF90089570E0B0
:10151000660F771F860F971FFC01858596850895B6
:1015200081E0613009F080E0089581E0633009F0E6
:1015300080E00895FC0186810895CF93DF93EC014C
:101540008C819D81DC01ED91FC910480F581E02D81
:101550006E8109951F86188A81E08A8B1E821B8AFC
:101560001C8A1D8A1E8A1F8A80E0DF91CF91089510
:101570002E9808952E9A08950F931F93CF93DF937B
:10158000D82FC62F8A010E94B80AD260DEBDF801AA
:101590008C2F882339F00DB407FEFDCF91919EBDAD
:1015A0008150F7CFC00FD12FD11D0DB407FEFDCF55
:1015B0000E94BA0ACE01DF91CF911F910F91089539
:1015C000CF93DF93C82FD62F0E94B80AC260CEBD3A
:1015D0000DB407FEFDCFDEBD0DB407FEFDCFDF91DC
:1015E000CF910C94BA0A9F92AF92BF92CF92DF92A2
:1015F000EF92FF920F931F93CF93DF936C01C42F51
:10160000D22F99249394E62EF12CEE0CFF1CE80EB9
:10161000F91E86E5E80EF11CA42EB12CABE2AA0E51
:10162000B11CAA0CBB1CAC0CBD1CF70180819181C4
:10163000DC01ED91FC910280F381E02D202F4D2FF4
:101640006C2F0995182F803EC9F5C1112BC061E0A0
:1016500088EE0E94E00A66E670E080E090E00E947A
:101660006C08F70180819181DC01ED91FC91019082
:10167000F081E02D202F4D2F6C2F0995182F8D30E4
:10168000D1F58FEF890D8330F8F0C11137C061E0DB
:1016900088EE0E94E00A66E670E080E090E00E943A
:1016A0006C081CC0F50180819181DC01ED91FC91F9
:1016B0000284F385E02D6D2F0995D3CF8D3061F431
:1016C0008FEF890D833050F464E670E080E090E0A5
:1016D0000E946C089394A9CF882319F2812FDF917F
:1016E000CF911F910F91FF90EF90DF90CF90BF901F
:1016F000AF909F900895882389F3C7CF8C2F90E0F7
:101700008B96880F991F8C0D9D1DFC018081918106
:10171000DC01ED91FC910284F385E02D6D2F09959C
:10172000DDCFCF93C82F0E94B80ACEBD0DB407FEFF
:10173000FDCF1EBC0DB407FEFDCF0E94BA0A8EB5C8
:10174000CF9108958F929F92AF92BF92CF92DF92E6
:10175000EF92FF920F931F93CF93DF93882E962ED5
:101760005A010E94DF066B017C0128E8C20E23E1CA
:10177000D21EE11CF11CC0E010E000E0D0E098288F
:101780000E94DF066C197D098E099F0997FF1EC014
:10179000692D80EF0E94E00A0E94DF066C197D0926
:1017A0008E099F0997FF09C088EC0E94910B87FF63
:1017B000F3CF60E888EC0E94E00A88EF0E94910B6A
:1017C000C82FCF70C43081F0CE30B9F08C2FDF91AC
:1017D000CF911F910F91FF90EF90DF90CF90BF902E
:1017E000AF909F908F9008950F5F1F4FA114B10489
:1017F00039F20A151B0521F6E9CFDF5FD33009F076
:10180000BFCFE4CFAF92BF92CF92DF92EF92FF9221
:101810000F931F93CF93DF93EC01B62EA42E690193
:101820000E94AA067C0186EDE114F10409F447C088
:10183000D701ED91FC91119787ED309709F43FC0E6
:1018400013969C9180E0981731F02081A21629F020
:1018500033968F5FF8CFF0E0E0E0D601ED93FC9394
:101860008BED309761F1228126952695203108F085
:101870002FE081E090E0A0E0B0E004C0880F991F65
:10188000AA1FBB1F2A95D2F70197F8019183808385
:101890006B2D80EE0E94E00A88ED0E94910BD7012B
:1018A00014969C91682F697F992329F0CA58DF4FBD
:1018B00068816260682B88ED0E94E00A80E0DF9119
:1018C000CF911F910F91FF90EF90DF90CF90BF903D
:1018D000AF90089588EC0E94910B85FF14C060E2E0
:1018E00088EC0E94E00A88EF0E94910B807C909126
:1018F00011018917E1F180931101803409F150F44D
:10190000882379F108958091EF03811130C064E05C
:1019100088EEE7CF803819F0803C09F1089588ED12
:101920000E94910B9091EF0381FD11C09230F9F06C
:1019300061EC88ED0E94E00A82E08093EF03089555
:1019400088ED0E94910B9091EF0381FDEFCF9330D2
:1019500071F063EC88ED0E94E00A83E0EECF81E055
:10196000ECCF61EC88ED0E94E00A1092EF0308953D
:10197000FC018789089570E0660F771F860F971F17
:10198000FC015687458781E00895482F80E1489FF4
:1019900090011124205E31092830310508F590911D
:1019A0009B029923E9F0892F90E0EDE9F2E061E0F4
:1019B00070E02191243078F0322F32953F7034134B
:1019C0000AC02F70DB0102C0AA0FBB1F2A95E2F7E5
:1019D0009D018A2B932BB2E0E33AFB0751F7089560
:1019E00090E080E0E2CFCF93DF93CDB7DEB72897CA
:1019F0000FB6F894DEBF0FBECDBFE22F29833A8326
:101A00004B835C836D837E838F83988720919B02B9
:101A10002E2B20939B02FE013396AE01475F5F4F52
:101A20002191243060F0ADE9B2E090E080E03D919A
:101A3000311111C085569D4FDC0112962C93E4178D
:101A4000F50771F728960FB6F894DEBF0FBECDBF2D
:101A5000DF91CF91089501968630910541F7EFCF40
:101A600080E00895089580E008952F923F924F926C
:101A70005F926F927F928F929F92AF92BF92CF921E
:101A8000DF92EF92FF920F931F93CF93DF937B012F
:101A90004A016901F901A080B180FB012180F901AF
:101AA00011821082FB01828160E181FD60E288EE9B
:101AB0000E94E00A3A2CA401F701608180E00E94B4
:101AC000A20B582EF6E08F17B1F381114EC088ECAF
:101AD0000E94910B82FF5DC080E30E94910B482E13
:101AE0008A151B0411F008F0432CF60180819181C6
:101AF0003501681A790A77FE02C0712C612CC42D59
:101B0000D0E0C615D7050CF43E01562C0E94B80A49
:101B1000F8E0FEBD0DB407FEFDCFF801552041F001
:101B20001EBC5A940DB407FEFDCF8EB58193F6CF3F
:101B3000060D171D0E94BA0A64E088EC0E94E00AB4
:101B4000F60180819181C80FD91FD183C0834214CF
:101B500020F0CA15DB0508F4AECF88EF0E94910B88
:101B6000F701928184FB91F99283852DDF91CF91CA
:101B70001F910F91FF90EF90DF90CF90BF90AF90AB
:101B80009F908F907F906F905F904F903F902F909D
:101B9000089580EF582EE9CF2F923F924F925F9297
:101BA0006F927F928F929F92AF92BF92CF92DF926D
:101BB000EF92FF920F931F93CF93DF93CDB7DEB7D2
:101BC00065970FB6F894DEBF0FBECDBF3C01342E33
:101BD000222E402EED8AEAA4FBA4188A1F861E86B8
:101BE0001D868E01035F1F4F9E01215F3F4F40E026
:101BF0000E94020C582E81111AC139822A824B820E
:101C00002D892C83DE82CD82B886AF82AE014F5FF4
:101C10005F4F68E080E20E94BC0A4D855E8560E00F
:101C200080E10E94A20B811120C1E114F10409F4AA
:101C300049C00F851889D80112968C91129737FEEA
:101C400047C0826012968C936501C114D10409F4D7
:101C500011C19C2D8D2D8C149D0410F4982D892D6F
:101C60009B878C874D855E856F85788987019E016E
:101C7000255F3F4FC3010E94350D582EB6E08B17EC
:101C800021F38111D4C0ECA5FDA53097A1F06B859F
:101C90007C850190F081E02D0190F081E02DC5015F
:101CA0008C199D099A8789879E01275F3F4FA7015D
:101CB0008CA59DA509958B859C85C81AD90A881580
:101CC000990518F64D855E8537FECBC080EACAC0FF
:101CD000816012968C93129711966C908FEF860DFF
:101CE000803408F0C4C02D843E840E94DF069B012E
:101CF000AC0128573C4E4F4F5F4F298B3A8B4B8B93
:101D00005C8BD80112968C9160E880FF60E488EECD
:101D10000E94E00A512C712C8114910409F476C0C0
:101D200063018614970408F46401CD8AA7016C2D21
:101D300080E10E94BC0A6C2D88E30E94E00AF80151
:101D40006081606280EF0E94E00A88EC0E94910B43
:101D500087FFFBCF60E888EC0E94E00A88EF0E94D2
:101D6000910B8F70582E412CB12CA12C552019F1BC
:101D70000E94DF0629893A894B895C89621B730BB3
:101D8000840B950B97FF17C036E05316E9F04EE031
:101D90005416B1F054E0551209C08FEFA81AB80AD2
:101DA0002114310489F02A143B0471F460E088E3C3
:101DB0000E94E00A2DC08C189D08EC0CFD1CACCFD5
:101DC000439493E0491691F360E088E30E94E00AAF
:101DD000D7016C9180E10E94E00A6D8988E30E943E
:101DE000E00AF8016081606280EF0E94E00A88ECFE
:101DF0000E94910B87FFFBCF60E888EC0E94E00A0D
:101E000088EF0E94910B8F70582EB0CF5110CECF1B
:101E100088EF0E94910BD80112969C91129785FB36
:101E200090F912969C934D855E855520D1F0852DB5
:101E300065960FB6F894DEBF0FBECDBFDF91CF9190
:101E40001F910F91FF90EF90DF90CF90BF90AF90D8
:101E50009F908F907F906F905F904F903F902F90CA
:101E6000089580E860E00E94A20B582EE0CF8AED32
:101E7000582EDDCF4D855E85552009F427CFD7CF6D
:101E80008F929F92AF92BF92CF92DF92EF920F9379
:101E90001F921F927F936F9388248394912CAA247E
:101EA000A394B12CD12CC12C42E0E42E00E029E017
:101EB00041E2FC016681848195810E94CC0D0F90E6
:101EC0000F900F900F900F91EF90DF90CF90BF90F9
:101ED000AF909F908F900895CF93DF931F92CDB7CF
:101EE000DEB789838091F804882339F0BE016F5FE3
:101EF0007F4F81EE94E00E94400F8091DE048823A2
:101F000039F0BE016F5F7F4F87EC94E00E94400F75
:101F10008091C404882339F0BE016F5F7F4F8DEA42
:101F200094E00E94400F8091AA04882339F0BE01FA
:101F30006F5F7F4F83E994E00E94400F0F90DF9125
:101F4000CF9108958F929F92AF92BF92CF92DF92DE
:101F5000EF920F93CF931F921F921F921F92912C7B
:101F6000812CB12CA12CD12CC12CE12C062F25E0E9
:101F700040E060E00E94CC0DC82F6CE271E080E090
:101F800090E00E946C080F900F900F900F908C2F94
:101F9000CF910F91EF90DF90CF90BF90AF909F9037
:101FA0008F9008958F929F92AF92BF92CF92DF92BF
:101FB000EF920F931F921F923F932F934A015A0162
:101FC000D12CC12CEE24E39400E026E040E80E94EE
:101FD000CC0D0F900F900F900F900F91EF90DF901E
:101FE000CF90BF90AF909F908F9008958F929F92C7
:101FF000AF92BF92CF92DF92EF920F931F931F92F7
:102000001F921F930F934A015A01D12CC12C32E029
:10201000E32E022F26E040E80E94CC0D0F900F9097
:102020000F900F901F910F91EF90DF90CF90BF9086
:10203000AF909F908F9008958F929F92AF92BF9292
:10204000CF92DF92EF920F93C42ED12C1F921F924A
:102050001F921F92912C812CB12CA12CE12C062FC8
:1020600021E043E2FC016285828193810E94CC0DD4
:102070000F900F900F900F900F91EF90DF90CF90F7
:10208000BF90AF909F908F9008958F929F92AF9244
:10209000BF92CF92DF92EF920F93C62ED12C1F9258
:1020A0001F925F934F9324E0822E912C34E0A32E55
:1020B000B12CE12C00E020E043EAFC016285828142
:1020C00093810E94CC0D0F900F900F900F900F9165
:1020D000EF90DF90CF90BF90AF909F908F9008953A
:1020E0008F929F92AF92BF92CF92DF92EF920F9317
:1020F000C42ED12C1F921F921F921F92912C812CC3
:10210000B12CA12CE12C062F23E043E2FC016285D7
:10211000828193810E94CC0D0F900F900F900F90B1
:102120000F91EF90DF90CF90BF90AF909F908F90E6
:102130000895CF92DF92FF920F931F93CF93DF9377
:1021400000D000D0CDB7DEB78C01F62E19821A82EE
:102150001B821C82462F61E10E941C104F2D60E102
:10216000C8010E941C104F2D64E0C8010E9470102D
:1021700083E0C82ED12CAE014F5F5F4F6F2DC80199
:102180000E944510811114C089819A81AB81BC8164
:102190009D7F83309140A041B10551F064E670E02D
:1021A00080E090E00E946C0881E0C81AD10819F71D
:1021B0004F2D64E1C8010E941C104F2D60E1C80141
:1021C0000E941C1064E170E080E090E00E946C08C6
:1021D0000F900F900F900F90DF91CF911F910F9163
:1021E000FF90DF90CF9008952F923F924F925F9291
:1021F0006F927F928F929F92AF92BF92CF92DF9217
:10220000EF92FF920F931F93CF93DF93CDB7DEB77B
:10221000E8970FB6F894DEBF0FBECDBFDC011A966B
:102220003C9131112CC1922E242E362E3C01FC0102
:10223000E280F380D701ED91FC910190F081E02DD7
:1022400060E0C70109958C01009709F41BC1FC01EE
:10225000C080D180C114D10409F417C15301F4E046
:10226000AF0EB11CDC011196BC92AE9214969C92FA
:10227000FE0131962F019F0148E050E060E0D3015C
:1022800012968D919C910E94D20F982EF801148283
:10229000811101C18D8191ED992E893059F5898087
:1022A000D701ED91FC910280F381E02D222D41E0D8
:1022B000632DC7010995F3018287882309F4E8C0DB
:1022C00098859583682F828193810E94A20F982E12
:1022D000D801CD92DC92882339F1D701ED91FC91A0
:1022E0000480F581E02DD3011A966C91C701099500
:1022F000F3011286892DE8960FB6F894DEBF0FBE63
:10230000CDBFDF91CF911F910F91FF90EF90DF90A4
:10231000CF90BF90AF909F908F907F906F905F9085
:102320004F903F902F900895811082C0950142E018
:10233000F3016285828193810E94C106982E8111EA
:102340008AC01F921F925F924F9258E0852E912C67
:1023500068E0A62EB12CD12CC12C79E2E72E00E04A
:1023600026E040EAF3016285828193810E94CC0DD0
:10237000982E0F900F900F900F9081116CC08B8151
:10238000D3011B968C931B97820120E048E050E01C
:102390001A966C911A9712968D919C910E94F60F45
:1023A000982E811158C04B815C8120E0F301628539
:1023B000828193810E94F60F982E81114CC0498131
:1023C00050E08E010F5D1F4F20E0D3011A966C91F3
:1023D0001A9712968D919C910E94F60F982E81115A
:1023E0003AC01F921F921F921F92912C812CB12CE8
:1023F000A12CE12C0E8129E040E0F301628582816D
:1024000093810E94CC0D982E0F900F900F900F90FB
:10241000811121C011E0D3011B968C911B9781176C
:1024200008F1412F68E0C3010E9470101F5FF3CFD5
:10243000482D413208F040E250E09201D3011A9653
:102440006C911A9712968D919C910E94D20F982EA2
:10245000882309F46BCF60E870E08CEB92E00E9477
:10246000160848CF1296ED91FC911397EA58FF4F4A
:1024700080818460808381E050968C933BCF49EDCE
:10248000942E38CF36ED932E35CF27ED922E32CFC6
:1024900084ED982E2FCFD182C0822CCF2F923F92E5
:1024A0004F925F926F927F928F929F92AF92BF9264
:1024B000CF92DF92EF92FF920F931F93CF93DF9310
:1024C000CDB7DEB7C358D1090FB6F894DEBF0FBE43
:1024D000CDBF3C01B62EA42E022FDC011496CD9068
:1024E000DC9060E870E08BEA91E00E941608F3014E
:1024F000868199EDF92E81110FC0108ED601ED91D4
:10250000FC910190F081E02D60E0C60109952C015D
:102510000097E9F4F6EDFF2E8F2DCD57DF4F0FB664
:10252000F894DEBF0FBECDBFDF91CF911F910F9109
:10253000FF90EF90DF90CF90BF90AF909F908F90E3
:102540007F906F905F904F903F902F900895FC0187
:10255000E080F180E114F10449F460E870E082EA7F
:1025600091E00E941608E7EDFE2ED6CF1301F7E0AA
:102570002F0E311CDC0111963C922E9214960C9376
:102580009E0126593F4F48E050E060E0F30184810E
:1025900095810E94D20F182F811199C2AB961FAD61
:1025A000AB97D201ED92FC92D601ED91FC910280A5
:1025B000F381E02D2A2D40E06B2DC6010995F30132
:1025C0008683882309F480C2E2969FADE2979087C4
:1025D000682F848195810E94A20FF82E882311F123
:1025E000D20114961C92D601ED91FC910480F581E4
:1025F000E02DD30116966C91C6010995F301168260
:1026000060E870E089E991E00E94160860E870E0F7
:102610008F2D0E94290A60E870E086E991E00E940F
:1026200016087ACF60E870E080E991E00E94160811
:1026300060E870E0D30116968C910E94290A60E848
:1026400070E08DE891E00E941608F2011482D60134
:10265000ED91FC910190F081E02DD30116966C91E3
:10266000C6010995009709F455CFFC010483910137
:1026700041E0D30116966C91169714968D919C911A
:102680000E94C1061111B9C0EC96BFADEC97EF9650
:10269000BFAFEF9760E870E089E891E00E9416080C
:1026A00060E870E0EF968FADEF970E94290A60E82E
:1026B00070E086E891E00E94160860E870E08EE61F
:1026C00091E00E9416082E01E1E44E0E511CC30158
:1026D0000296CE57DF4F99838883C258D040D201EB
:1026E0005096EE96BFAFAEAFEE97EF96FFADEF9779
:1026F000FF1509F4AFC0EFE1F1E0D2011196FC93B0
:10270000EE93CE57DF4F88819981C258D0401396FF
:102710009C938E93129714961C92149719961C9260
:1027200019971A961C921A971D961C921D971F9620
:102730001C921E921E9790961C92909791961C92B6
:10274000919792961C92929798961C929897EE96D3
:10275000EEADFFADEE971696FC93EE931597189697
:10276000FC93EE9317971C96FC93EE931B97D30163
:1027700014960D90BC91A02DC158DF4FB983A8834A
:10278000CF57D040F301F681CF57DF4FF883C158C0
:10279000D0408E010F5F1F4F2F2D49E050E06F2F6B
:1027A000CD010E94F60F811121C0AB80BC805F92E9
:1027B0004F921F930F9360E4862E912CD12CC12C45
:1027C00072E0E72E0F2D26E040E8CF57DF4F6881FB
:1027D000C158D040C158DF4F88819981CF57D04030
:1027E0000E94CC0D0F900F900F900F90D301529636
:1027F0008C91823079F1F39478CF133108F012E1A3
:10280000412F50E09E0126593F4FF301668184819C
:1028100095810E94D20F182F882309F435CF60E8E4
:1028200070E087ED90E00E941608F12E60E870E0FD
:102830008F2D0E94290A60E870E081EF90E00E94ED
:102840001608D301ED91FC910480F581E02DC301C0
:10285000099562CE60E870E086E691E00E94160875
:1028600060E870E0F30182890E94290A60E870E064
:1028700083E691E00E941608D30152968C915297FC
:1028800021EDF22E823091F6910142E016966C9184
:10289000169714968D919C910E94C10660E870E095
:1028A0008EE591E00E94160860E870E0F3018785EC
:1028B0000E94290A60E870E08BE591E00E9416080A
:1028C00068EE73E080E090E00E946C081F921F9217
:1028D0001F921F92912C812CB12CA12CD12CC12C98
:1028E000E12CD3011F960C911F9729E040E016962A
:1028F0006C91169714968D919C910E94CC0DF82E98
:102900000F900F900F900F908111D7C068EE73E079
:1029100080E090E00E946C0860E870E080E591E063
:102920000E94160860E870E0F30180890E94290A7D
:1029300060E870E08DE491E00E94160860E870E0C5
:1029400082E491E00E94160860E870E0D30151969D
:102950008C910E94290A60E870E08FE391E00E9468
:10296000160860E870E082E391E00E94160860E8D3
:1029700070E080E00E94290A60E870E08FE291E058
:102980000E9416081F921F921F921F92F301018D41
:102990002BE041E26681848195810E94CC0D182F45
:1029A00060E870E080E291E00E94160860E870E064
:1029B000812F0E94290A60E870E08DE191E00E9479
:1029C00016080F900F900F900F90112319F01530EB
:1029D00009F02BCF1F921F921F921F92912C812CD6
:1029E000B12CA12CD12CC12CE12C00E02AE041E239
:1029F000D30116966C91169714968D919C910E9416
:102A0000CC0D182F60E870E082E191E00E9416087A
:102A100060E870E0812F0E94290A60E870E08FE092
:102A200091E00E9416080F900F900F900F901123C5
:102A300019F0153009F0F9CEFE01EF5BFF4F85E28A
:102A400091E091838083FF93EF93CE0101969F9352
:102A50008F9330E4832E912C40E8A42EB12CD12CFE
:102A6000C12C52E2E52E00E026E041E8F301668148
:102A7000848195810E94CC0D182F60E870E087E07A
:102A800091E00E94160860E870E0812F0E94290AF8
:102A900060E870E084E091E00E94160860E870E071
:102AA00084EF90E00E94160881E0D30157968C9342
:102AB0000F900F900F900F902FCD60E870E086EE92
:102AC00090E00E941608B2CE84EDF82E25CDF201DA
:102AD000F182E082A4CE8F929F92AF92BF92CF926A
:102AE000DF92EF92FF920F931F93CF93DF9300D06B
:102AF00000D0CDB7DEB77C01C62ED42E59014801D7
:102B00001C821B821A8219828E010F5F1F4F9E0149
:102B10002D5F3F4F0E94020C182F882309F445C0F7
:102B200061E870E087EA95E00E94160861E870E0CD
:102B3000812F0E94290A61E870E084EA95E00E94F2
:102B4000160861E870E082E895E00E94160861E8E6
:102B500070E08C2D0E94290A61E870E08FE795E013
:102B60000E94160861E870E08FE595E00E94160863
:102B700061E870E08D2D0E94290A61E870E08CE523
:102B800095E00E941608812F0F900F900F900F90E4
:102B9000DF91CF911F910F91FF90EF90DF90CF9039
:102BA000BF90AF909F908F90089549815A816B811B
:102BB0007C8184019501C7010E94350D182FE3CF58
:102BC0002F923F924F925F926F927F928F929F923D
:102BD000AF92BF92CF92DF92EF92FF920F931F932B
:102BE000CF93DF93CDB7DEB768970FB6F894DEBF0B
:102BF0000FBECDBF1B8A38E03C8B3CE33D8B8A3F48
:102C00003FEF9307D9F416ED812F68960FB6F8942D
:102C1000DEBF0FBECDBFDF91CF911F910F91FF900F
:102C2000EF90DF90CF90BF90AF909F908F907F906C
:102C30006F905F904F903F902F900895222E642EBA
:102C4000362E7C01DC0116960D911C911797CE0152
:102C5000439617969C938E9316971A962C939E01E3
:102C60002F5F3F4F42E150E060E0C7010E94D20F6A
:102C7000782EF70117830683182F8111C5CF498459
:102C80005A848B849C84FD81FF8B3E81388F670141
:102C900086E5C80ED11C56011E8AD5018D919D91E5
:102CA0005D010097D1F5BE89BF5FBE8BB031A9F73A
:102CB000F601819191916F01009709F06EC07394B4
:102CC000F0E17F12F5CFF7018681978117ED892B0F
:102CD00009F49ACF2286262D40E0632DC7010E9479
:102CE0005506082F14ED882309F48ECF682FC701ED
:102CF0000E94AA06009709F486CFDC0114962C9254
:102D0000602FC7010E94A20F182F882309F47CCFDF
:102D1000602FC7010E94330677CFDC01ED91FC9153
:102D20000084F185E02D09958111BDCFF5019291C7
:102D300082918F01DC01ED91FC910088F189E02DF9
:102D4000688D0995882309F4AECFF80180819181BF
:102D5000DC01ED91FC910484F585E02DA401B20124
:102D60000995882361F0022D262D432D6E89C70118
:102D70000E94F30A182F813D09F495CF45CFF80141
:102D800080819181DC01ED91FC910684F785E02D35
:102D90006F8909958111E7CF86CFDC01ED91FC9118
:102DA0000084F185E02D0995811189CFF60192917A
:102DB00082918F01DC01ED91FC910088F189E02D79
:102DC000688D099581110DC0022D262D432D672D8B
:102DD000C7010E94F30A182F877F813D09F014CFA5
:102DE0006ECFF80180819181DC01ED91FC9104842A
:102DF000F585E02DA401B2010995811160CFF8019C
:102E000080819181DC01ED91FC910684F785E02DB4
:102E10006F8909958823C1F252CFCF92DF92EF924A
:102E2000FF921F93CF93DF93EC01162F7A01FA01E3
:102E300080819181A281B3818130F3E09F07F1E02D
:102E4000AF07B105C9F170F48115E1E09E07AE0747
:102E5000B10509F450C081309140A140B10561F144
:102E600080E041C0833021E0920720E1A207B10554
:102E700029F083309340A041B10591F7412F64E1DF
:102E8000CE010E941C10412F60E1CE010E941C1057
:102E900064E170E080E090E00E946C086A85F701D0
:102EA0002181269521706770412F8A819B810E9424
:102EB000E0151092A302D4CF8091A3028111D0CF4C
:102EC000412F61E1CE010E941C10412F60E1CE0133
:102ED0000E941C10412F64E0CE010E94701081E01E
:102EE0008093A30281EBDF91CF911F91FF90EF9030
:102EF000DF90CF900895462F61E1CE010E941C1013
:102F0000412F60E1CE010E941C101092A3028A851D
:102F100087701770880F880F880F182B09F4A0CFBF
:102F2000EA80FB806701F6E5CF0ED11CD0E0C0E05F
:102F3000D6018D919D916D010097C1F0DC01ED915D
:102F4000FC910084F185E02D099518130FC0AB9614
:102F5000CC0FDD1FCE0DDF1D88819981DC01ED9145
:102F6000FC910480F581E02D09957ACF2196C0313E
:102F7000D105F1F675CFCF92DF92EF92FF920F93CA
:102F80001F93CF93DF93CDB7DEB72E970FB6F8948C
:102F9000DEBF0FBECDBFFC012089211111C010E0A2
:102FA000812F2E960FB6F894DEBF0FBECDBFDF91F6
:102FB000CF911F910F91FF90EF90DF90CF900895E8
:102FC0007C010E94DF06F70104851585268537857B
:102FD000601B710B820B930B97FDE1CF81E090E0BA
:102FE0009E878D878E010F5F1F4F9E01235F3F4F8E
:102FF00041E06285828193810E946B15182F8111B7
:1030000021C082E0D82E01E089818D2139F1198615
:103010001A861B861C86AE01475F5F4F602FC70173
:103020000E944510C82E811119C0AE01475F5F4F45
:10303000602FC7010E940D17813B19F0882371F0A2
:10304000C82E1C2D0E94DF066C597F4F8F4F9F4F5B
:10305000F7016487758786879787A2CFDD0C0F5F9E
:10306000083091F601E0F7018385801758F319863F
:103070001A861B861C86AE01475F5F4F602FC70113
:103080000E944510D82E811117C089859A858770B6
:1030900091708130914081F48B859C8581609C8703
:1030A0008B87AE01475F5F4F602FC7010E940D17EE
:1030B000813B29F0811102C00F5FD5CFD82E1D2D85
:1030C000C1CF0F931F93CF93DF938091E90390912A
:1030D000E803892B809386029091E703992389F076
:1030E000892B80938602E7E8F2E02EE832E080E068
:1030F000919191118F5F2E173F07D1F78111109297
:10310000E703E091E503F091E6033097B1F1028027
:10311000F381E02D86E892E009958091E40382FF37
:103120002CC080FF04C081E595E00E944803D0E0F8
:10313000C0E00BE415E08091E40380FF0EC0FE01C7
:10314000EA57FD4F80811F928F931F930F930E9428
:10315000E1030F900F900F900F902196C830D1058A
:1031600051F78091E40380FF08C089E495E0DF9186
:10317000CF911F910F910C944803DF91CF911F9134
:103180000F9108951092E803E6E8F2E011821282AE
:10319000138214821582168217820C9461180F9381
:1031A0001F93CF93DF93CDB7DEB7AA970FB6F894EE
:1031B000DEBF0FBECDBF8091DF02882309F427C197
:1031C0001091E9001F708091EC0080FF39C080E809
:1031D000182B1092E9008091E80083FF15C1E7EDFC
:1031E000F2E08FED92E02091F10021938E179F077E
:1031F000D1F78091D802833009F470C018F581307E
:1032000009F447C0823009F4B3C08091E80083FF1D
:10321000EDC08091D7029091D8029A3008F0E6C0B4
:10322000E92FF0E0EA5EF64E0C94E527C919EF1994
:10323000F619EF19F619511A731AF6196F1B7C1B40
:1032400080E0C6CF8A3009F482C08B3009F463C0B5
:103250008930D9F68091D7028132B9F68091DB02AC
:103260009091DC02892B89F68091E800877F80931A
:10327000E8008091E80082FF2CC08091F1008093EB
:10328000CB028091E8008B778093E8000E94FF04D6
:10329000BCCF8091D702813A09F0B7CF8091E80086
:1032A000877F8093E8008091DB029091DC02892B7C
:1032B00061F060E090E080E070E00E947104809135
:1032C000E8008B778093E800A0CF68E08CEC92E078
:1032D000F3CF8091DF028111CCCF97CF8091D702BD
:1032E000813A09F092CF8091DB029091DC02892B28
:1032F00009F08BCF8091E800877F8093E800809170
:10330000E80080FFFCCF809110018093F100809154
:10331000E8008E77B9CF8091D702813209F075CF5E
:103320008091DB029091DC02892B09F06ECF8091B5
:10333000E800877F8093E8000E94FF048091D90213
:10334000809310011092E9030E94C2185ECF809111
:10335000D702813209F059CF8091E800877F8093AE
:10336000E8000E94FF048091DA028093CA024DCFE8
:103370008091D702813A09F048CF8091E800877F99
:103380008093E8008091E80080FFFCCF8091CA0222
:10339000BCCF803889F0823849F58091DB028F708C
:1033A000873020F58093E9008091EB0085FB88272A
:1033B00080F91092E90006C08091D4029091D50264
:1033C000911182609091E800977F9093E80080933C
:1033D000F1001092F1008091E8008E7731C0282F23
:1033E0002D7F21F48823F1F0823079F18091E8007B
:1033F00083FF0AC08091E800877F8093E800809176
:10340000EB0080628093EB001F701093E900AA9696
:103410000FB6F894DEBF0FBECDBFDF91CF911F91E5
:103420000F9108958091D902813001F7933009F00E
:1034300080E08093D5021092E9008091E800877FB8
:103440008093E8000E94FF04D1CF8091D9028111BE
:10345000F2CF8091DB028F702FEF280F263030F6ED
:103460008093E9002091EB0020FFE5CF933031F409
:103470008091EB0080628093EB00DDCF9091EB00B8
:1034800090619093EB0021E030E001C0220F8A951B
:10349000EAF72093EA001092EA008091EB0088603E
:1034A000EACF8111A3CF0091D9020F778091E30079
:1034B0008078802B8093E3008091E800877F809361
:1034C000E8000E94FF048091E80080FFFCCF80911B
:1034D000E30080688093E30083E0011101C082E093
:1034E0008093DF0283CF8058823008F07FCF209115
:1034F000D9023091DA022C3D83E03807A1F583E050
:103500008A838AE289834FB7F894DE01139620E01C
:103510003EE051E2E32FF0E050935700E49120FFAA
:1035200003C0E295EF703F5FEF708E2F90E0EA30BE
:10353000C0F0C7968D939D932F5F243159F74FBFED
:103540008091E800877F8093E8006AE270E0CE0116
:1035500001960E9471048091E8008B778093E800C7
:1035600045CFC096E7CF4091DB025091DC02832F1C
:1035700099278330910509F440C070F58130910599
:1035800009F46BC0029709F031CF8BE390E0E2E9D8
:10359000F3E02091E800277F2093E8002091DD02EE
:1035A0003091DE028217930708F49C0140E0211558
:1035B000310509F061C041115FC08091E80082FDD2
:1035C000CACF8091DF02882331F2853021F28091C9
:1035D000E80083FFF2CFBFCF8132910591F18232B3
:1035E000910509F003CF4115510509F440C0E0E30E
:1035F000F3E04130510569F2F9CE3327213031052E
:10360000C1F060F02230310509F0F0CEEFEDF3E0CB
:10361000E4918E2F90E0EFEDF3E007C0E7E2F4E0F5
:10362000E4918E2F90E0E7E2F4E0009709F4DECE1B
:10363000B0CFEDE1F4E0E4918E2F90E0EDE1F4E025
:10364000F4CF4115510571F089E090E0EDEBF3E026
:103650004130510509F49DCFC9CE82E190E0EDECF7
:10366000F3E097CF89E090E0E4EAF3E092CF80E4E2
:1036700090E0E2E5F3E08DCF8091DF02882309F44A
:103680006ACF853009F467CF8091E80083FD63CF6E
:103690008091E80082FD91CF8091E80080FF87CF84
:1036A0008091F3009091F2008927982789272115AE
:1036B000310519F08830910550F041E0089709F084
:1036C00040E08091E8008E778093E80070CF4491CD
:1036D0004093F1003196215031090196E8CF8038AE
:1036E00009F084CE8091E800877F8093E800809184
:1036F000D6028093F1006FCE811178CE0091D9026D
:10370000023008F073CE8091E800877F8093E80054
:103710000093D6020E94FF04002371F084E080939E
:10372000DF0242E061EC81E00E941E0546E261ECAE
:1037300083E00E941E055ACE8091E30087FDEECF04
:1037400081E0EDCFCF93DF932091E2023091E3024D
:103750002817390701F19093E3028093E202E09188
:10376000E503F091E6033097B1F0EC010084F185B8
:10377000E02D09958091E4038570853061F4DF9335
:10378000CF9389E394E09F938F930E94E1030F907E
:103790000F900F900F90DF91CF910895CF93DF930B
:1037A0002091E0023091E1022817390701F190934E
:1037B000E1028093E002E091E503F091E6033097A7
:1037C000B1F0EC010680F781E02D09958091E403CA
:1037D0008570853061F4DF93CF938BE294E09F9303
:1037E0008F930E94E1030F900F900F900F90DF9145
:1037F000CF910895AF92BF92CF92DF92EF92FF9256
:103800000F931F93CF936091910470919204409114
:103810008504509186042091790430917A04809136
:103820006D0490916E04E0919902F0919A026E17E6
:103830007F07B1F4E0919702F0919802E417F50741
:1038400079F4E0919502F0919602E217F30741F4C2
:10385000E0919302F0919402E817F90709F45FC030
:1038600070939A0260939902509398024093970242
:103870003093960220939502909394028093930242
:1038800088E0EBE9F2E0DF011D928A95E9F72091EB
:10389000890430918A0440918B0450918C0460918A
:1038A0008D0470918E0480918F04909190040E94F9
:1038B000F30C20917D0430917E0440917F0450915F
:1038C00080046091810470918204809183049091BE
:1038D00084040E94F30C2091710430917204409191
:1038E0007304509174046091750470917604809112
:1038F0007704909178040E94F30C20916504309134
:103900006604409167045091680460916904709165
:103910006A0480916B0490916C040E94F30C0E94E5
:10392000FE067C010E946A0C8091EF03813009F44D
:103930005EC008F460C0823029F0833009F463C0AF
:10394000C0E017C0C0E080914004807F803189F4DE
:103950000E94DF0668537F4F8F4F9F4F60938E0208
:1039600070938F02809390029093910280E28093F3
:10397000400481E5C82E85E0D82E91E7A92E95E078
:10398000B92E8601F801819191918F01009739F04C
:10399000DC01ED91FC910680F781E02D0995A016E0
:1039A000B10681F780914004803409F4B8C068F50D
:1039B000803209F49EC0803309F4ABC0813109F034
:1039C00042C010927105F601819191916F010097AB
:1039D00039F0DC01ED91FC910480F581E02D099531
:1039E000C016D10681F782E1809340042CC083E1A8
:1039F00080934004A5CF80914004807F803109F4FA
:103A00009FCF81E1F5CFC1E09ECF813509F49AC007
:103A1000803809F4AAC08035B1F488EC0E94910B7B
:103A200086FF11C081E5809340040E94DF066C5040
:103A30007E4F8F4F9F4F60938E0270938F028093C3
:103A40009002909391022FB7F8948091EA0390919D
:103A5000EB03A091EC03B091ED032FBF8E199F09EA
:103A60008536910560F09F938F9388EC90E09F934B
:103A70008F930E94E1030F900F900F900F90809111
:103A8000400490919202981749F1809392021F92FC
:103A90008F9387EB90E09F938F930E94E1030F90A9
:103AA0000F900F900F90809192028039B9F480911D
:103AB000EF03823009F069C082E191E09F938F9318
:103AC0008CEA90E09F938F930E94E1030E9446044A
:103AD0000E946C0F0F900F900F900F9081E0CF918C
:103AE0001F910F91FF90EF90DF90CF90BF90AF901C
:103AF00008950E94DF0600918E0210918F0220919E
:103B0000900230919102601B710B820B930B97FD19
:103B10009ACF61E088EE0E94E00A80E465CF88EEEB
:103B20000E94910B80FD8FCF60E488EC0E94E00A38
:103B300088ED0E94910B682F686088ED0E94E00A72
:103B400080E552CF0E94DF0600918E0210918F0215
:103B50002091900230919102601B710B820B930BAC
:103B600097FD71CF80E8809340042C2F40E060E007
:103B70008BEF94E00E94E015882329F0823D09F440
:103B800062CF80EA31CF80E92FCF87E191E096CFF5
:103B9000FF920F931F93CF93DF9300D000D01F921B
:103BA000CDB7DEB74983952F5A836B837C838D8392
:103BB0002C813D8181E02115310531F05F3F19F401
:103BC00081E04F3F09F080E080FD83C281E0232B3C
:103BD00031F09F3F19F481E04F3F09F080E02B81E5
:103BE00080FD78C0692F70E050E0CB01E4E0880FE1
:103BF000991FEA95E1F78C519D4FDC01A40FB51F89
:103C0000222309F45BC01C9280E090E1899FF001BF
:103C10001124E60FF71F34E0EE0FFF1F3A95E1F78E
:103C2000E40FF51FE75BFB4FE49180E48E0F8032D9
:103C300008F046C0E05CFF0BEE0FFF1FE75BFA4F9A
:103C400085919491FC011E2F8F2F82958F70823069
:103C500008F4F0C08E3009F03CC2E1113AC22223D0
:103C600009F437C21092E9030E94C2189FEF20E7BF
:103C700082E0915020408040E1F700C000000E94A7
:103C80005204F89487E797E790930108809300081F
:103C900087E090EBDC018093720590937305A0930D
:103CA0007405B093750588E19CE00FB6F894A8956B
:103CB000809360000FBE90936000FFCF8C91A5CFE2
:103CC000EF3B58F4E83A48F5E53AD0F4E430B0F484
:103CD000E13089F0F0E0E0E0B6CFE83E38F4E03ED5
:103CE00068F4EF3BB9F7E0E0F0EEADCFE03F90F3E2
:103CF000F0E0F065A8CFE1E0F0E0A5CFF0E0A3CFE1
:103D0000E53A29F0E63A31F4E2E8F0E49CCFE1E864
:103D1000F0E499CFE3E8F0E496CFE83A09F445C03F
:103D2000E93A09F445C0EA3A09F445C0EB3A09F426
:103D300045C0EC3A09F445C0ED3A09F445C0EE3A05
:103D400009F445C0EF3A09F445C0E13B09F445C028
:103D5000E03B09F445C0E23B09F445C0E33B09F40C
:103D600045C0E43B09F445C0E53B09F445C0E63BEA
:103D700009F445C0E73B09F445C0E83B09F445C0F8
:103D8000E93B09F445C0EA3B09F445C0EB3B09F4C3
:103D900045C0EC3B09F445C0ED3B09F445C0EE3BA2
:103DA00009F045C0E0E7F4E44ECFE2EEF4E44BCF97
:103DB000E9EEF4E448CFEAEEF4E445CFE5EBF4E4D1
:103DC00042CFE6EBF4E43FCFE3EBF4E43CCFE4EBAB
:103DD000F4E439CFE7EBF4E436CFECECF4E433CFA2
:103DE000EDECF4E430CFE3E8F5E42DCFEAE8F5E4D8
:103DF0002ACFE2E9F5E427CFE4E9F5E424CFE1E2D4
:103E0000F6E421CFE3E2F6E41ECFE4E2F6E41BCFD2
:103E1000E5E2F6E418CFE6E2F6E415CFE7E2F6E4F1
:103E200012CFEAE2F6E40FCFEFE6F4E40CCFE0E0E5
:103E3000F4E409CF8F2F8F70F82E8F2F807F19F029
:103E4000F29480EFF822222309F4E7C0FF2039F032
:103E50008091E8038F298093E8030E946118112361
:103E600009F437C18EE7810F833070F5123831F1D4
:103E7000133839F511E003E50E944604812309F067
:103E800028C1802F0E942D040E9461189FEF21EE0F
:103E900084E0915020408040E1F700C00000802F76
:103EA0000E9421040F900F900F900F900F90DF91C0
:103EB000CF911F910F91FF900C94611812E009E3CC
:103EC000DBCF14E007E4D8CF8CEF810F813A20F4E8
:103ED000812F0E942D04E6CF80E2810F883068F4A4
:103EE000177021E030E001C0220F1A95EAF78091A7
:103EF000E903822B8093E903D5CF8BE5810F8330D3
:103F0000B0F481E890E0153A31F082E890E0163A9A
:103F100011F083E890E00F900F900F900F900F90AA
:103F2000DF91CF911F910F91FF900C94CE1B88E5EC
:103F3000810F873108F0CDC082EE90E0183A09F485
:103F400060C089EE90E0193A09F45BC08AEE90E017
:103F50001A3A09F456C085EB90E01B3A09F451C0B7
:103F600086EB90E01C3A09F44CC083EB90E01D3ADC
:103F700009F447C084EB90E01E3A09F442C087EB95
:103F800090E01F3AF1F18CEC90E0113BD1F18DEC17
:103F900090E0103BB1F183E891E0123B91F18AE8A7
:103FA00091E0133B71F182E991E0143B51F184E916
:103FB00091E0153B31F181E292E0163B11F183E291
:103FC00092E0173BF1F084E292E0183BD1F085E2F9
:103FD00092E0193BB1F086E292E01A3B91F087E261
:103FE00092E01B3B71F08AE292E01C3B51F08FE6BD
:103FF00090E01D3B31F080E790E01E3B11F090E037
:1040000080E00F900F900F900F900F90DF91CF9165
:104010001F910F91FF900C94A21B112309F18EE7C1
:10402000810F833068F5123829F1133831F511E02A
:1040300003E50E944604812399F0802F0E942D04FD
:104040000E9461189FEF21EE84E091502040804053
:10405000E1F700C00000802F0E9421040E94611837
:10406000FF20B9F18F2D80959091E80389238093EB
:10407000E80318CF12E009E3DCCF14E007E4D9CF5E
:104080008CEF810F813A10F4812FE6CF80E2810F0F
:10409000883070F4177021E030E001C0220F1A95CB
:1040A000EAF720959091E90329232093E903D6CFDD
:1040B0008BE5810F833028F490E080E00E94CE1BD6
:1040C000CFCF185A173160F690E080E00E94A21B13
:1040D000C7CF0F900F900F900F900F90DF91CF915F
:1040E0001F910F91FF900895EF92FF920F931F93EE
:1040F000CF93DF932091DF022430B1F521E02093AC
:10410000E90021E8215021F03091E80035FF33C06B
:104110002091E80025FF28C0C92FD82F0E94D00485
:10412000811114C00D2F1C2F88E0E82EF12C8091F6
:10413000E80085FD27C08091E8008E778093E80035
:104140000E94CF180E94D004882389F38091E80050
:104150008E778093E80088E0ED2FFC2FACECB2E086
:1041600001900D928A95E1F7DF91CF911F910F9108
:10417000FF90EF900895EFE3F1E03197F1F700C081
:104180000000C0CFF80181918F018093F100F1E030
:10419000EF1AF10861F6DACFAF92BF92CF92DF92B9
:1041A000EF92FF920F931F93CF93DF936C01CB019C
:1041B000E22EDB01ED91FC910084F185E02D099563
:1041C0001F928F9382EB92E09F938F930E94E10363
:1041D000E801E00EF12EF11C0F900F900F900F9060
:1041E0008CEAA82E82E0B82ECE15DF0561F0899109
:1041F0001F928F93BF92AF920E94E1030F900F9096
:104200000F900F90F1CF89EA92E09F938F930E94D5
:10421000E1030F900F90F8018281813099F48FE8CB
:1042200092E09F938F930E94E1030F900F90DF9194
:10423000CF911F910F91FF90EF90DF90CF90BF90A3
:10424000AF900895D601129688E001900D928A955C
:10425000E1F70E94DF06D6011B967C936E931A97B6
:10426000E6CF5F926F927F928F929F92AF92BF92B2
:10427000CF92DF92EF92FF920F931F93CF93DF9332
:1042800000D0CDB7DEB77C016DB67EB6DC015796A7
:104290008C91811119C0512C852D0FB6F8947EBEDA
:1042A0000FBE6DBE0F900F90DF91CF911F910F91B8
:1042B000FF90EF90DF90CF90BF90AF909F908F9046
:1042C0007F906F905F9008950E94DF06F701038949
:1042D000148925893689601B710B820B930B97FD1E
:1042E000DACFADB6BEB661E870E080E892E00E9439
:1042F000160881E890E00E94040861E870E08DE70C
:1043000092E00E94160861E870E08AE492E00E9460
:10431000160861E870E0D7011A968C910E94290A6C
:1043200061E870E087E492E00E94160861E870E0BE
:1043300080E192E00E94160861E870E0F701838551
:104340000E94290A61E870E08DE092E00E94160860
:10435000D7011B968C9190E08134910508F056C0EE
:104360009A83898389819A81EDB7FEB7E81BF90B9F
:104370000FB6F894FEBF0FBEEDBF2DB73EB72F5F4F
:104380003F4F690189019E012F5F3F4FD7011A9668
:104390004C911A9716966C91169714968D919C9144
:1043A0000E946B15582E811134C029813A81233027
:1043B000310598F1F70185859685009749F0DC0174
:1043C000ED91FC910190F081E02D40E0B70109955D
:1043D00089819A8110E0892B09F479C029813A8179
:1043E000812F90E08217930708F069C08C0D9D1D06
:1043F00060E870E0DC018C910E94290A60E870E0BE
:1044000088EB91E00E9416081F5FE8CF80E490E0FF
:10441000A7CFB4E08B1709F45AC061E870E08BEFC6
:1044200091E00E94160861E870E0852D0E94290A3B
:1044300061E870E088EF91E00E941608511047C0D3
:1044400089819A81892B09F442C060E870E087ED88
:1044500091E00E94160889809A800CE010E0C40167
:10446000002E02C0969587950A94E2F7982F9F70C8
:1044700080E3890F8A3310F087E3890F60E870E0EA
:104480000E94FE07045011090C3FEFEF1E0739F799
:1044900060E870E084ED91E00E94160860E870E04A
:1044A0008DEB91E00E94160880E890E00E940408DD
:1044B00060E870E08AEB91E00E94160889CF232B18
:1044C00031F060E870E085EB91E00E9416080FB6CD
:1044D000F894BEBE0FBEADBE0E94DF06F701208D70
:1044E000620F711D811D911D638B748B858B968B63
:1044F000D3CECF931092F3031092F20388EE93E0A1
:10450000A0E0B0E08093F4039093F503A093F6034A
:10451000B093F7038FE491E09093F1038093F0035D
:104520008FEF9FEF9093FD038093FC0387E791E06B
:104530009093FC048093FB041092030581E0809328
:104540000405109205058DEF94E090930205809389
:1045500001051092FD0488E08093FE048CE38093B3
:10456000FF0410920005EBEFF4E0C1E08DEF94E062
:104570001586C687178694878387359625E0E634A7
:10458000F207B1F71092710581E18093400481EE4A
:1045900094E00E94EA0387EC94E00E94EA038DEA2B
:1045A00094E00E94EA0383E994E00E94EA0381E830
:1045B00091E0909388048093870490937C04809387
:1045C0007B049093700480936F04909364048093B1
:1045D000630481E691E090935304809352048BEF3F
:1045E00094E09093550480935404109262041092C6
:1045F000560488E0809357049CE390935804C0933A
:10460000590480935A0484E080935B0410925C0404
:1046100010925D0410925E0410925F041092600488
:1046200010926104A1E5B5E0FD0190E080E02191E8
:104630003191232B09F044C0880F991FFC01EF5AD8
:10464000FA4F82E594E09183808381E691E0909334
:104650004204809341048BEF94E090934404809350
:104660004304109251041092450488E0809346045C
:104670009CE39093470491E090934804809349040D
:1046800084E080934A0410924B0410924C041092E0
:104690004D0410924E0410924F041092500490E07A
:1046A00080E02D913D91232B89F4880F991FFC0107
:1046B000EF5AFA4F81E494E091838083CF9108957B
:1046C00001968031910509F0B2CFBFCF01968031BC
:1046D000910539F7F3CF1F920F920FB60F92112465
:1046E0008F939F93AF93BF938091EE03811113C07B
:1046F0008091EA039091EB03A091EC03B091ED035C
:104700004196A11DB11D8093EA039093EB03A09302
:10471000EC03B093ED03BF91AF919F918F910F90F8
:104720000FBE0F901F9018951F920F920FB60F9209
:1047300011242F933F934F935F936F937F938F93A6
:104740009F93AF93BF93EF93FF938091E10082FF1C
:1047500009C08091E20082FF05C08091E1008B7F5B
:104760008093E1008091DA0080FF1FC08091D80023
:1047700080FF1BC08091DA008E7F8093DA008091E9
:10478000D90080FFA1C080E189BD82E189BD09B463
:1047900000FEFDCF81E08093DF028091C80281118D
:1047A00004C00E9452040E9450058091E10080FFE5
:1047B00021C08091E20080FF1DC08091E2008E7FC9
:1047C0008093E2008091E20080618093E20080911A
:1047D000D80080628093D80019BC85E08093DF0206
:1047E0008091CB028093C9021092CB021092E90310
:1047F0000E94C2188091E10084FF2FC08091E200E6
:1048000084FF2BC080E189BD82E189BD09B400FE2F
:10481000FDCF8091D8008F7D8093D8008091E100FA
:104820008F7E8093E1008091E2008F7E8093E20092
:104830008091E20081608093E2008091D60288231B
:1048400009F448C084E08093DF021092E9030E94DB
:10485000C2188091C9028093CB028091E10083FF4E
:1048600022C08091E20083FF1EC08091E100877F1B
:104870008093E10082E08093DF021092D602809163
:10488000E1008E7F8093E1008091E2008E7F809333
:10489000E2008091E20080618093E20042E060E00B
:1048A00080E00E941E05FF91EF91BF91AF919F9113
:1048B0008F917F916F915F914F913F912F910F90C9
:1048C0000FBE0F901F90189519BC1092DF02109226
:1048D000C8026BCF8091E30087FD02C081E0B3CFB7
:1048E00083E0B1CFCF93DF93CDB7DEB72A970FB672
:1048F000F894DEBF0FBECDBF84B7877F84BF0FB6ED
:10490000F894A8958091600088618093600010926F
:1049100060000FBE80E890E00FB6F89480936100CD
:10492000909361000FBE8AEF97E09093850180938A
:10493000840186E091E09093E6038093E5038BE0A9
:1049400093E00E9448030E9452040E94500578940C
:1049500082E084BD93E095BD9AEF97BD80936E0091
:104960008091E40381608093E403269A0E94BA0A4E
:10497000219A229A2398209A80E58CBD81E08DBDF2
:10498000259868E188E80E94E00A60E288E70E94D2
:10499000E00A60E088E70E94E00A10E000E088E6B4
:1049A0000E94910B0F5F1F4F80FF1CC061EC88EDD0
:1049B0000E94E00A60E280ED0E94E00A64E088EE76
:1049C0000E94E00A88EE0E94910B82FFFBCF0E94BA
:1049D0006A0C60E288EC0E94E00A61E080E80E94D4
:1049E000E00A03C00F3F1007D1F687E894E09093E8
:1049F000EF048093EE048BE794E09093D5048093CA
:104A0000D4048FE694E09093BB048093BA0483E6C9
:104A100094E09093A1048093A0048091DF028430FD
:104A200009F0C0C00E94EB06882309F4BBC089EFDF
:104A300092E00E9448038BEE92E00E9448033324E8
:104A40003A9423E0222E30EE632E32E0732E48E1BA
:104A5000842E912C8091DF02853009F4A6C00E943B
:104A6000FA1B06EA12E0512C852D0E94C50C5C0150
:104A7000F801C080D1808C159D0571F1412CEE2488
:104A8000E394F12CCA24DB24C6018E219F21892BBB
:104A9000E9F04E825F8221E0C5018E219F21892BA2
:104AA00009F420E028870E94FE068160782F9A870B
:104AB00089874E815F8168858A850E94C81DF801BB
:104AC000808191818E259F25918380834394EE0C74
:104AD000FF1CF0E14F12D8CF53940E5F1F4F80E1BF
:104AE0005812C2CF39823A821B820E94FE06816030
:104AF000782F9D838C8349815A816B818D810E949F
:104B0000C81D0E9446049091A5028917B9F00E9421
:104B100046048093A5029091E4039570953051F47A
:104B20001F928F937F926F920E94E1030F900F90DC
:104B30000F900F908091A5020E946C0F2091E400CD
:104B40003091E5008091C6029091C702281739077D
:104B500031F18091E4009091E5009093C702809339
:104B6000C6020E94EB068823D1F08091DF028430D8
:104B7000B1F48091E9008F709091EC0090FD4FC0EE
:104B800090E0892B2092E9009091EB0090FF04C007
:104B90009091EE0097FD61C08F708093E9000E94B4
:104BA000CF1858CF0E94CF1838CF8091DF028430C1
:104BB00011F11092EE0380E40FB6F894A89580925C
:104BC00060000FBE8093600083B7817F846083BFE5
:104BD00083B7816083BF7894889583B78E7F83BFC6
:104BE0000FB6F894A895809160008861809360006A
:104BF000109260000FBE8091D502882369F00E9458
:104C0000FA1B10E0812F0E94C50C892B09F049C0C6
:104C10001F5F1031B9F71ECF0E94FA1B1BCF90E81F
:104C2000B0CFE0910101F0910201E90FF11D208167
:104C30009F5F309105019323909304012093F1002D
:104C40009091E80095FD09C09091E80090FF05C0A3
:104C50009091E8009E779093E80090910401209154
:104C60000301291721F02091E80025FDDACF2091DA
:104C7000F3009091F200322F292F232B09F48CCFCF
:104C80009091E80090FF88CF9091E80095FD06C0D4
:104C90009091E8009E779093E8007ECF1092F1000B
:104CA000F3CFE0E1E9BDF2E1F9BD09B400FEFDCFCB
:104CB0008091D8008F7D8093D8008091E000826041
:104CC0008093E0008091E00081FDFCCFC3CE78941A
:104CD0001F920F920FB60F9211248F939F93AF9351
:104CE000BF938091EA039091EB03A091EC03B09104
:104CF000ED030196A11DB11D8093EA039093EB0390
:104D0000A093EC03B093ED03BF91AF919F918F916E
:104D10000F900FBE0F901F9018950E94FE2608F46A
:104D200081E008950E942A2788F09F5798F0B92FB4
:104D30009927B751B0F0E1F0660F771F881F991FD0
:104D40001AF0BA95C9F714C0B13091F00E94442707
:104D5000B1E008950C944427672F782F8827B85F17
:104D600039F0B93FCCF3869577956795B395D9F728
:104D70003EF490958095709561957F4F8F4F9F4F32
:104D80000895E89409C097FB3EF49095809570953E
:104D900061957F4F8F4F9F4F9923A9F0F92F96E987
:104DA000BB279395F695879577956795B795F111FC
:104DB000F8CFFAF4BB0F11F460FF1BC06F5F7F4F99
:104DC0008F4F9F4F16C0882311F096E911C07723AB
:104DD00021F09EE8872F762F05C0662371F096E8B4
:104DE000862F70E060E02AF09A95660F771F881F83
:104DF000DAF7880F9695879597F90895990F000827
:104E0000550FAA0BE0E8FEEF16161706E807F9079C
:104E1000C0F012161306E407F50798F0621B730B37
:104E2000840B950B39F40A2661F0232B242B252BB8
:104E300021F408950A2609F4A140A6958FEF811D5B
:104E4000811D089557FD9058440F551F59F05F3F3D
:104E500071F04795880F97FB991F61F09F3F79F09C
:104E600087950895121613061406551FF2CF46951E
:104E7000F1DF08C0161617061806991FF1CF8695A0
:104E80007105610508940895E894BB276627772784
:104E9000CB0197F908950E94FE2608F48FEF08953C
:104EA0000E9463270C94D4270E94C62738F00E94E2
:104EB000CD2720F0952311F00C94BD270C94C32727
:104EC00011240C9445270E94222770F3959FC1F36B
:104ED000950F50E0551F629FF001729FBB27F00DA8
:104EE000B11D639FAA27F00DB11DAA1F649F6627FD
:104EF000B00DA11D661F829F2227B00DA11D621F4C
:104F0000739FB00DA11D621F839FA00D611D221F05
:104F1000749F3327A00D611D231F849F600D211DE9
:104F2000822F762F6A2F11249F5750409AF0F1F06C
:104F300088234AF0EE0FFF1FBB1F661F771F881FD5
:104F400091505040A9F79E3F510580F00C94BD2729
:104F50000C9445275F3FE4F3983ED4F3869577950C
:104F60006795B795F795E7959F5FC1F7FE2B880F7B
:104F7000911D9695879597F9089597F99F6780E811
:104F800070E060E008959FEF80EC089500240A949B
:104F90001616170618060906089500240A94121614
:104FA0001306140605060895092E0394000C11F447
:104FB000882352F0BB0F40F4BF2B11F460FF04C0F4
:104FC0006F5F7F4F8F4F9F4F0895EE0FFF1F05902C
:0A4FD000F491E02D0994F894FFCF4E
:104FDA000586010000FFB4057420B305B105B205CA
:104FEA0001FF66756C6C006C6F770000000000E5CD
:104FFA000800000000280A000000004E12330D9D30
:10500A000A31219A0A320D300D950A900A870ABB95
:10501A000CB80C4B0AFEFF00007D0A00000000D508
:10502A0008BB08DC08DB08E208DF08DF080000002C
:10503A0000F410330DB705BB17DE059910300DD9F2
:10504A0005DD0600000000AA06550633060000002A
:04505A0000CC200066
:00000001FF
